:10000000011C00A1010101011C000100010101010D
:100010001C000101010101011C610100011C011C06
:100020001C012100011D1D1D1C6101007B1D011D06
:100030001C0121017B011D011C6101001D011D012D
:100040001C000100010101E11C61011C1D1D1D1DA1
:100050001C0101071D09217D1C611D091D01091DD0
:100060001C011D1D1D1D1BBD1C001D091D1D1D7D11
:100070000101011B7B0501011C00F501011B0100B1
:100080000101010101051D1DE107F5E101FD1D1D36
:1000900001A1E7E101011BE101010101A1E7A1E7E4
:1000A000011D091D010101000101FD1DFD1D1D9D19
:1000B000011D1D01010101011DE11D1DFDFD051DAC
:1000C00001010101011D1D1D05000001E11C617BF5
:1000D000001C01017B0101010161E701011B01E13C
:1000E0001C716101E1010101A0E10501E30301E1EE
:1000F0001D1D1D1D1D1D1D1D001C1B0101151D1D90
:100100001C001D1BBD1C617B7B1501011D1D010118
:1001100000A001A01C0001A0A1B5011B1D091D1D0F
:100120001C00151D1D1C617B1C611701E10501E10F
:10013000001C01011D01011B010101FD1D1D1D1DF3
:1001400001011D09211D0121010109010161E76171
:1001500061FB6765011C6161611C1B1D1D1D1D1D6F
:100160001C1CA1A1151DFD1D017B007B1D1D1DFD7E
:100170001C1D0101BB0501610161000169017101E3
:100180001C1D01010105071D011C0101E11C0101EC
:100190001C1D010101BBA0017B1C0101FD1DFD1DFA
:1001A000001CA101BB61071D017B111D1D011D016B
:1001B000010009011D1DA0BB7B1C616103011D1D08
:1001C000001DA0A1071B01017B1C0101057707E1B0
:1001D000001DA0A1A71B81016101611DFBE11C00A5
:1001E000001DA101A107FBE01C7B1D1D1D7D7D1DC8
:1001F0001CBB1C001C00131D001C00017B7161E175
:10020000001D01B1A71BBBB1A0171503011D1D1DCA
:100210001C71617161716101001D01B1A7FBB1A188
:10022000013B01000101211D001D0101010121010E
:10023000011B012075670561013B01017B01211D47
:10024000001D010101012101201D05B70577011DD8
:10025000013B1C1D01012101001D010101012101C2
:10026000207DA77D1D25011D013B1D1D01012101D3
:10027000001D010101012101201D1D1D7C1D1DE12D
:100280001CA1A1BB7517011D0101FB67671D157D31
:100290001D0101010101151D01071DEF01410100B3
:1002A000011C610161676100BB010101FBA10161EA
:1002B0001C0161770101E11B01611D0801217D081D
:1002C0000001610101010101FC61716105611177AA
:1002D00015011D016901710171611D1D7501611B10
:1002E000717B0101011D7D011D1D00010001010146
:1002F0001D01000100010101010D1D011B01E109AA
:1003000001290115604991610101010101E1011B10
:100310000101010101010000011D1D1D1D1DBD1D6B
:100320001D1D1D1D1D1D1D017BBDE7BDE7BD07BDBD
:1003300007BD07BD07BD07BD07BD07BDE7BD07BDBD
:1003400007BD070101BD07BD071D1D1D1DFD1D1DAD
:10035000FD03111D1D1D9D1D1D1D1D1D1DBD07BD69
:1003600007BD071DE7011DFD1D1D1D1B1D1D1D1DBD
:100370001DBD071D1D1D1DBD171D1D1D1D1D1D1D89
:10038000011D1D1D011D1D1D1D1D1D1D1D1D1D1DD5
:100390001D1D1D09091D1D1D1D1D1D1D1D7D1D1D55
:1003A0001D7D111D7D65071D1D111D1D1D1D1DA917
:1003B00065091D671D67031D051D1D1D1D1D1D1CD8
:1003C0007D1D093D1D7D111D7D1D1D23011D1D1D53
:1003D0007D7D1D67A705177D7D1D031D1D05071D5F
:1003E000011D1D1D157D017D7B7D017D7D1D1D1D5B
:1003F0001D1D7D1D1D1D7D11BD7D7D7D1D1D1D1DB9
:10040000011C00A1010101011C0001000101010109
:100410001C000101010101011C610100011C011C02
:100420001C012100011D1D1D1C6101007B1D011D02
:100430001C0121017B011D011C6101001D011D0129
:100440001C000100010101E11C61011C1D1D1D1D9D
:100450001C0101071D09217D1C611D091D01091DCC
:100460001C011D1D1D1D1BBD1C001D091D1D1D7D0D
:100470000101011B7B0501011C00F501011B0100AD
:100480000101010101051D1DE107F5E101FD1D1D32
:1004900001A1E7E101011BE101010101A1E7A1E7E0
:1004A000011D091D010101000101FD1DFD1D1D9D15
:1004B000011D1D01010101011DE11D1DFDFD051DA8
:1004C00001010101011D1D1D05000001E11C617BF1
:1004D000001C01017B0101010161E701011B01E138
:1004E0001C716101E1010101A0E10501E30301E1EA
:1004F0001D1D1D1D1D1D1D1D001C1B0101151D1D8C
:100500001C001D1BBD1C617B7B1501011D1D010114
:1005100000A001A01C0001A0A1B5011B1D091D1D0B
:100520001C00151D1D1C617B1C611701E10501E10B
:10053000001C01011D01011B010101FD1D1D1D1DEF
:1005400001011D09211D0121010109010161E7616D
:1005500061FB6765011C6161611C1B1D1D1D1D1D6B
:100560001C1CA1A1151DFD1D017B007B1D1D1DFD7A
:100570001C1D0101BB0501610161000169017101DF
:100580001C1D01010105071D011C0101E11C0101E8
:100590001C1D010101BBA0017B1C0101FD1DFD1DF6
:1005A000001CA101BB61071D017B111D1D011D0167
:1005B000010009011D1DA0BB7B1C616103011D1D04
:1005C000001DA0A1071B01017B1C0101057707E1AC
:1005D000001DA0A1A71B81016101611DFBE11C00A1
:1005E000001DA101A107FBE01C7B1D1D1D7D7D1DC4
:1005F0001CBB1C001C00131D001C00017B7161E171
:10060000001D01B1A71BBBB1A0171503011D1D1DC6
:100610001C71617161716101001D01B1A7FBB1A184
:10062000013B01000101211D001D0101010121010A
:10063000011B012075670561013B01017B01211D43
:10064000001D010101012101201D05B70577011DD4
:10065000013B1C1D01012101001D010101012101BE
:10066000207DA77D1D25011D013B1D1D01012101CF
:10067000001D010101012101201D1D1D7C1D1DE129
:100680001CA1A1BB7517011D0101FB67671D157D2D
:100690001D0101010101151D01071DEF01410100AF
:1006A000011C610161676100BB010101FBA10161E6
:1006B0001C0161770101E11B01611D0801217D0819
:1006C0000001610101010101FC61716105611177A6
:1006D00015011D016901710171611D1D7501611B0C
:1006E000717B0101011D7D011D1D00010001010142
:1006F0001D01000100010101010D1D011B01E109A6
:1007000001290115604991610101010101E1011B0C
:100710000101010101010000011D1D1D1D1DBD1D67
:100720001D1D1D1D1D1D1D017BBDE7BDE7BD07BDB9
:1007300007BD07BD07BD07BD07BD07BDE7BD07BDB9
:1007400007BD070101BD07BD071D1D1D1DFD1D1DA9
:10075000FD03111D1D1D9D1D1D1D1D1D1DBD07BD65
:1007600007BD071DE7011DFD1D1D1D1B1D1D1D1DB9
:100770001DBD071D1D1D1DBD171D1D1D1D1D1D1D85
:10078000011D1D1D011D1D1D1D1D1D1D1D1D1D1DD1
:100790001D1D1D09091D1D1D1D1D1D1D1D7D1D1D51
:1007A0001D7D111D7D65071D1D111D1D1D1D1DA913
:1007B00065091D671D67031D051D1D1D1D1D1D1CD4
:1007C0007D1D093D1D7D111D7D1D1D23011D1D1D4F
:1007D0007D7D1D67A705177D7D1D031D1D05071D5B
:1007E000011D1D1D157D017D7B7D017D7D1D1D1D57
:1007F0001D1D7D1D1D1D7D11BD7D7D7D1D1D1D1DB5
:00000001FF
